BL51 BANKED LINKER/LOCATER V6.02                                                        10/16/2011  00:43:52  PAGE 1


BL51 BANKED LINKER/LOCATER V6.02, INVOKED BY:
C:\KEIL\C51\BIN\BL51.EXE Spot_Welder.obj TO Spot_Welder


INPUT MODULES INCLUDED:
  Spot_Welder.obj (SPOT_WELDER)


LINK MAP OF MODULE:  Spot_Welder (SPOT_WELDER)


            TYPE    BASE      LENGTH    RELOCATION   SEGMENT NAME
            -----------------------------------------------------

            * * * * * * *   D A T A   M E M O R Y   * * * * * * *
            REG     0000H     0008H     ABSOLUTE     "REG BANK 0"

            * * * * * * *   C O D E   M E M O R Y   * * * * * * *
            CODE    0000H     01ABH     ABSOLUTE     



SYMBOL TABLE OF MODULE:  Spot_Welder (SPOT_WELDER)

  VALUE           TYPE          NAME
  ----------------------------------

  -------         MODULE        SPOT_WELDER
  N:000AH         SYMBOL        ARCOUNT
  D:00F0H         SYMBOL        B
  C:002BH         SYMBOL        BEGIN
  C:00B7H         SYMBOL        CK_KEY
  C:008BH         SYMBOL        CK_PEDAL
  N:0024H         SYMBOL        COMP
  C:0056H         SYMBOL        COM_0
  N:0022H         SYMBOL        COUNT
  B:00B0H.6       SYMBOL        CP
  C:0091H         SYMBOL        DEB0
  C:009EH         SYMBOL        DEB3
  C:009FH         SYMBOL        DEB4
  B:0020H.2       SYMBOL        DIGIT
  C:0126H         SYMBOL        DNH
  C:0137H         SYMBOL        DN_DO
  C:0141H         SYMBOL        DN_RET
  C:00D3H         SYMBOL        DOV
  C:011BH         SYMBOL        DO_DN
  C:0142H         SYMBOL        DO_UD
  C:00F4H         SYMBOL        DO_UP
  B:00A8H.7       SYMBOL        EA
  B:00B0H.2       SYMBOL        FIRE
  N:0020H         SYMBOL        FLAGS
  C:019FH         SYMBOL        FONT
  C:0059H         SYMBOL        FRONT
  B:0020H.4       SYMBOL        HWAVE
  C:0185H         SYMBOL        IND
  C:015DH         SYMBOL        IND1
  C:016FH         SYMBOL        IND2
  C:017BH         SYMBOL        IND3
BL51 BANKED LINKER/LOCATER V6.02                                                      10/16/2011  00:43:52  PAGE 2


  C:0182H         SYMBOL        IND4
  C:0152H         SYMBOL        INDIC
  B:00B0H.2       SYMBOL        INT0
  B:00B0H.3       SYMBOL        INT1
  N:000FH         SYMBOL        KEYARR
  N:0046H         SYMBOL        KEYDA
  N:0005H         SYMBOL        KEYDB
  N:0026H         SYMBOL        KEYDBT
  N:0007H         SYMBOL        KEYFARR
  N:0027H         SYMBOL        KEYTM
  B:00B0H.3       SYMBOL        KEY_DN
  B:00B0H.4       SYMBOL        KEY_UP
  C:0047H         SYMBOL        MAIN
  N:0063H         SYMBOL        MAXTIME
  N:0001H         SYMBOL        MINTIME
  C:00E6H         SYMBOL        ND
  C:00D8H         SYMBOL        NDN
  C:0075H         SYMBOL        NEG
  C:00E8H         SYMBOL        NP
  C:00E2H         SYMBOL        NUD
  C:00DDH         SYMBOL        NUP
  C:016AH         SYMBOL        NZ
  B:0020H.0       SYMBOL        ON_OFF
  D:0090H         SYMBOL        P1
  D:00B0H         SYMBOL        P3
  B:00B0H.5       SYMBOL        PED_IN
  N:0025H         SYMBOL        PED_ST
  B:0020H.1       SYMBOL        PRESS
  N:0028H         SYMBOL        PREV
  C:00A7H         SYMBOL        PULSE
  C:00B2H         SYMBOL        REF1
  C:00B0H         SYMBOL        REF2
  C:0066H         SYMBOL        REF_1
  C:006DH         SYMBOL        REF_2
  C:0078H         SYMBOL        REF_3
  N:0029H         SYMBOL        REPCNT
  B:00B0H.0       SYMBOL        RXD
  B:00B0H.1       SYMBOL        SCAN0
  B:00B0H.0       SYMBOL        SCAN1
  B:0090H.2       SYMBOL        SEG_A
  B:0090H.3       SYMBOL        SEG_B
  B:0090H.4       SYMBOL        SEG_C
  B:0090H.5       SYMBOL        SEG_D
  B:0090H.6       SYMBOL        SEG_E
  B:0090H.7       SYMBOL        SEG_F
  B:00B0H.7       SYMBOL        SEG_G
  C:0083H         SYMBOL        SUBR
  B:00B0H.4       SYMBOL        T0
  B:00B0H.5       SYMBOL        T1
  N:0031H         SYMBOL        TENS
  N:0021H         SYMBOL        TIME
  B:00B0H.1       SYMBOL        TXD
  C:0080H         SYMBOL        T_OFF
  C:014FH         SYMBOL        UD_OFF
  C:0151H         SYMBOL        UD_RET
  C:016CH         SYMBOL        UN
  N:0030H         SYMBOL        UNITS
BL51 BANKED LINKER/LOCATER V6.02                                                      10/16/2011  00:43:52  PAGE 3


  C:00FFH         SYMBOL        UPH
  C:0110H         SYMBOL        UP_DO
  C:011AH         SYMBOL        UP_RET
  C:00EDH         SYMBOL        W1
  C:00F3H         SYMBOL        W2
  C:00AEH         SYMBOL        WAIT_6MS
  N:0023H         SYMBOL        ZERO
  C:0000H         LINE#         58
  C:0003H         LINE#         60
  C:000BH         LINE#         62
  C:0013H         LINE#         64
  C:001BH         LINE#         66
  C:0023H         LINE#         68
  C:002BH         LINE#         73
  C:002DH         LINE#         74
  C:0030H         LINE#         75
  C:0033H         LINE#         76
  C:0036H         LINE#         77
  C:0039H         LINE#         78
  C:003CH         LINE#         79
  C:003DH         LINE#         80
  C:003FH         LINE#         81
  C:0041H         LINE#         82
  C:0043H         LINE#         83
  C:0045H         LINE#         84
  C:0047H         LINE#         86
  C:0049H         LINE#         87
  C:004BH         LINE#         88
  C:004CH         LINE#         89
  C:004EH         LINE#         90
  C:0051H         LINE#         91
  C:0054H         LINE#         92
  C:0056H         LINE#         93
  C:0059H         LINE#         94
  C:005CH         LINE#         95
  C:005EH         LINE#         96
  C:0061H         LINE#         97
  C:0064H         LINE#         98
  C:0066H         LINE#         99
  C:0069H         LINE#         100
  C:006BH         LINE#         101
  C:006DH         LINE#         102
  C:0070H         LINE#         103
  C:0073H         LINE#         104
  C:0075H         LINE#         105
  C:0078H         LINE#         106
  C:007AH         LINE#         107
  C:007CH         LINE#         108
  C:007EH         LINE#         109
  C:0080H         LINE#         110
  C:0083H         LINE#         111
  C:0085H         LINE#         112
  C:0087H         LINE#         113
  C:0089H         LINE#         114
  C:008BH         LINE#         117
  C:008DH         LINE#         118
  C:008FH         LINE#         119
BL51 BANKED LINKER/LOCATER V6.02                                                      10/16/2011  00:43:52  PAGE 4


  C:0091H         LINE#         120
  C:0093H         LINE#         121
  C:0095H         LINE#         122
  C:0097H         LINE#         123
  C:0099H         LINE#         125
  C:009BH         LINE#         126
  C:009CH         LINE#         127
  C:009EH         LINE#         141
  C:009FH         LINE#         142
  C:00A1H         LINE#         143
  C:00A2H         LINE#         144
  C:00A4H         LINE#         145
  C:00A6H         LINE#         146
  C:00A7H         LINE#         148
  C:00A9H         LINE#         149
  C:00ABH         LINE#         150
  C:00ADH         LINE#         151
  C:00AEH         LINE#         153
  C:00B0H         LINE#         154
  C:00B2H         LINE#         155
  C:00B4H         LINE#         156
  C:00B6H         LINE#         157
  C:00B7H         LINE#         160
  C:00B9H         LINE#         161
  C:00BBH         LINE#         162
  C:00BDH         LINE#         163
  C:00BFH         LINE#         164
  C:00C1H         LINE#         165
  C:00C2H         LINE#         166
  C:00C4H         LINE#         167
  C:00C5H         LINE#         168
  C:00C6H         LINE#         169
  C:00C7H         LINE#         170
  C:00C9H         LINE#         171
  C:00CBH         LINE#         172
  C:00CDH         LINE#         173
  C:00CFH         LINE#         174
  C:00D1H         LINE#         175
  C:00D3H         LINE#         176
  C:00D6H         LINE#         177
  C:00D8H         LINE#         178
  C:00DBH         LINE#         179
  C:00DDH         LINE#         180
  C:00E0H         LINE#         181
  C:00E2H         LINE#         182
  C:00E4H         LINE#         183
  C:00E6H         LINE#         184
  C:00E8H         LINE#         185
  C:00EAH         LINE#         186
  C:00EDH         LINE#         188
  C:00EFH         LINE#         189
  C:00F1H         LINE#         190
  C:00F3H         LINE#         191
  C:00F4H         LINE#         195
  C:00F7H         LINE#         196
  C:00FAH         LINE#         197
  C:00FDH         LINE#         198
BL51 BANKED LINKER/LOCATER V6.02                                                      10/16/2011  00:43:52  PAGE 5


  C:00FFH         LINE#         199
  C:0101H         LINE#         200
  C:0103H         LINE#         201
  C:0104H         LINE#         202
  C:0107H         LINE#         203
  C:0109H         LINE#         204
  C:010BH         LINE#         205
  C:010DH         LINE#         206
  C:0110H         LINE#         207
  C:0112H         LINE#         208
  C:0114H         LINE#         209
  C:0116H         LINE#         210
  C:0118H         LINE#         211
  C:011AH         LINE#         212
  C:011BH         LINE#         216
  C:011EH         LINE#         217
  C:0121H         LINE#         218
  C:0124H         LINE#         219
  C:0126H         LINE#         220
  C:0128H         LINE#         221
  C:012AH         LINE#         222
  C:012BH         LINE#         223
  C:012EH         LINE#         224
  C:0130H         LINE#         225
  C:0132H         LINE#         226
  C:0134H         LINE#         227
  C:0137H         LINE#         228
  C:0139H         LINE#         229
  C:013BH         LINE#         230
  C:013DH         LINE#         231
  C:013FH         LINE#         232
  C:0141H         LINE#         233
  C:0142H         LINE#         237
  C:0145H         LINE#         238
  C:0148H         LINE#         239
  C:014AH         LINE#         240
  C:014DH         LINE#         241
  C:014FH         LINE#         242
  C:0151H         LINE#         243
  C:0152H         LINE#         246
  C:0155H         LINE#         247
  C:0158H         LINE#         248
  C:015BH         LINE#         249
  C:015DH         LINE#         250
  C:015FH         LINE#         251
  C:0162H         LINE#         252
  C:0163H         LINE#         253
  C:0165H         LINE#         254
  C:0168H         LINE#         255
  C:016AH         LINE#         256
  C:016CH         LINE#         257
  C:016FH         LINE#         258
  C:0172H         LINE#         259
  C:0174H         LINE#         260
  C:0175H         LINE#         261
  C:0177H         LINE#         262
  C:0179H         LINE#         263
BL51 BANKED LINKER/LOCATER V6.02                                                      10/16/2011  00:43:52  PAGE 6


  C:017BH         LINE#         264
  C:017DH         LINE#         265
  C:017EH         LINE#         266
  C:0180H         LINE#         267
  C:0182H         LINE#         268
  C:0184H         LINE#         269
  C:0185H         LINE#         271
  C:0187H         LINE#         272
  C:0189H         LINE#         273
  C:018AH         LINE#         274
  C:018CH         LINE#         275
  C:018DH         LINE#         276
  C:018FH         LINE#         277
  C:0190H         LINE#         278
  C:0192H         LINE#         279
  C:0193H         LINE#         280
  C:0195H         LINE#         281
  C:0196H         LINE#         282
  C:0198H         LINE#         283
  C:0199H         LINE#         284
  C:019BH         LINE#         285
  C:019CH         LINE#         286
  C:019EH         LINE#         287
  -------         ENDMOD        SPOT_WELDER

******************************************************************************
* RESTRICTED VERSION WITH 0800H BYTE CODE SIZE LIMIT; USED: 0187H BYTE (19%) *
******************************************************************************

Program Size: data=8.0 xdata=0 code=427
LINK/LOCATE RUN COMPLETE.  0 WARNING(S),  0 ERROR(S)
